:09FD46000126000128000129003A
:10FB880012F8A812FD9812FE01D294E526B4FF13CC
:10FB9800E546D39400400CD54609E4F5437F0AFEB8
:10FBA80012FDD330080812FCE1C208E4F54620B083
:10FBB8000620080312F9E00526E529B401C8052442
:10FBC800E524D394FA40BFE4F5240530E53070020B
:10FBD800052F12FE01D3E5309458E52F940240A674
:10FBE8007F7712FD6BE4F532E42532FFE434EEFE54
:10FBF80074082532F8E6FD12FCA90532E532C394F3
:10FC08001440E57D557F167EEE12FCA9759F808015
:01FC1800FEED
:10FCA9008E3C8F3D8D3E12FE0175F65575F6AA758F
:10FCB900F65575BF04853EF6E53CF5F4853DF575C9
:10FCC900F7807B007A00793FAF3DAE3C12FDC7E576
:08FCD9003FB53E02D322C32215
:10F8A800D2947580FF43BF027B007A0079227F00E3
:10F8B8007EEE12FDC7AD22E4FFFE12FDFA7B007A50
:10F8C8000079237F017EEE12FDC7AD237F017E0004
:10F8D80012FDFA7B007A00792D7F027EEE12FDC7B9
:10F8E800AD2D7F027E0012FDFA7B007A00792E7F13
:10F8F800037EEE12FDC7AD2E7F037E0012FDFA7B5C
:10F90800007A00792C7F047EEE12FDC7AD2C7F04AF
:10F918007E0012FDFA7B007A00792A7F057EEE12BE
:10F92800FDC7AD2A7F057E0012FDFA7B007A0079BB
:10F93800487F067EEE12FDC7AD487F067E0012FDA9
:10F94800FA7B007A0079317F077EEE12FDC7AD3170
:10F958007F077E0012FDFA7B007A0079257F087EFA
:10F96800EE12FDC7AD257F087E0012FDFA7B007AF6
:10F978000079277F097EEE12FDC7AD277F097E003B
:10F9880012FDFA7D237F0B7E0012FDFA7B007A00C0
:10F99800792B7F107EEE12FDC7AD2B7F107E0012F3
:10F9A800FDFAE52B7026752901FB7A0079347F165C
:10F9B8007EEE12FDC7E534B4551212FE01E4FD7F58
:10F9C800167EEE12FCA943BF0202020075804CD2DB
:08F9D800A0C2A1C2A2C2A32239
:04FE0100759FA72220
:0BFDD300EF1FAC0670011E4C70F62202
:10FD4F000141FF014B0101430001429601490001AE
:08FD5F004400014C00014800C2
:10FD9800C292E4F543C208E5486003B4FF0375481E
:02FDA800FE2239
:0BFDDE00C292E4F543C2087542962271
:09FDE900D2927F0A7E0002FDD3D4
:10F9E000E4F520D2097F04FE12FDD3C209A2B09231
:10F9F00000D2097F037E0012FDD3C209A2B092019A
:10FA0000D2097F037E0012FDD3C209A2B09202D2B6
:10FA1000097F037E0012FDD3C209A2B09203D2096E
:10FA20007F037E0012FDD3C209A2B09204D2097FE7
:10FA3000037E0012FDD3C209A2B09205D2097F0352
:10FA40007E0012FDD3C209A2B09206D2097F037EC6
:10FA50000012FDD3C209A2B09207D209E543C394B4
:10FA600096500AAF430543744F2FF8A620C209E50C
:10FA700043B54204D2088056E5436407704278508B
:10FA8000E6FDB4061808E6FE08E67A002400FFEA60
:10FA90003EFEEF640A4E700575420C8031ED640342
:10FAA00060077850E6FFB406057542088020EFB481
:10FAB00010097855E62409F5428013754296800EA8
:10FAC000E543B403097850E6B41903754206754658
:01FAD0000233
:01FAD1002212
:07FD1900744F2536F8E6FFE8
:10FD20007E15D209C2B1DEFEE4FDEF1392B1EFC33E
:10FD300013FF7E12DEFE0DBD08F0D2B17F087E00FB
:05FD400012FDD3C20911
:01FD4500229B
:10FCE10012F4BF501312FDE912FDF212F6BE5005D7
:10FCF10012F08D800302FDDE12FDDEE541B4011735
:10FD0100E4FD7F107EEE12FCA9AD487F067EEF1266
:08FD1100FCA9759F8080FE2211
:10F4BF00E54365426002C322784FE6FFF4600AEF2E
:10F4CF0065486005EF6002C3227850E66419600357
:10F4DF0002F564FB7A00794F7D0412FC668E338F40
:10F4EF00347853E6FE08E67C002400FFEC3EFEEF86
:10F4FF0065347003EE65336002C3227852E6FF185D
:10F50F00E6FEC39F40028002AF067852E6FDEEC3CF
:10F51F009D400518E6FE8002AE05E548C39F4006F4
:10F52F00E548D39E4002C322AF267E0012FC5B1239
:10F53F00FC197C007D2812FAFDED2404F536E4F564
:10F54F0035E535C39536500B7F327E0012FDD3055E
:10F55F003580EED3227850E6FF6403600CEF64062B
:10F56F006007EF64106002C3227851E6FE08E67C64
:10F57F00002400FFEC3EFEEF640A4E600302F68BA0
:10F58F007850E66403707A12FC197C007D0512FA3C
:10F59F00FD8D4AE54A6401603A054CE54C75F0056E
:10F5AF0084E5F0702CF54C754A0112FC197C007D36
:10F5BF002812FAFDED2404F536E4F535E535C3954B
:10F5CF0036400302F68B7F327E0012FDD305358065
:10F5DF00EBC322AF267E0012FC5B12FC197C007D70
:10F5EF002812FAFDED2404F536E4F535E535C3951B
:10F5FF0036400302F68B7F327E0012FDD305358035
:10F60F00EB7850E664067074FB7A007937FFFE12D0
:10F61F00FDBA7B007A0079387F017E0012FDBA7B3C
:10F62F00007A0079397F027E0012FDBA7B007A00E2
:10F63F00793A7F037E0012FDBA7855E6B537100888
:10F64F00E6B5380B08E6B5390608E6653A6002C339
:10F65F0022AF267E0012FC5B12FC197C007D281263
:10F66F00FAFDED2404F536E4F535E535C39536504E
:10F67F000B7F327E0012FDD3053580EE7B007A00C2
:10F68F00794FE54224FEFD12FC668E338F34744DA4
:10F69F002542F8E6FE744E2542F8E67C002400FF72
:0EF6AF00EC3EFEEFB53406EEB53302D322C3B7
:01F6BD00222A
:10F08D00E4F5367850E6B40617E4F536E536C39563
:10F09D0042400302F2BE12FD1912FE01053680EC4C
:10F0AD007850E66403600302F20108E6FE08E67C90
:10F0BD00002400F534EC3EF5337854E6F535784F01
:10F0CD00E6FF12FD20784FE6FF12FD837850E6FF34
:10F0DD0012FD207850E6FF12FD83E534640A4533B6
:10F0ED007012E53525E02404FF12FD20E53525E0FD
:10F0FD002404800CE53525E0FF12FD20E53525E0E3
:10F10D00FF12FD83E536C39535400302F19DE4FF03
:10F11D0012FD20E4FF12FD83E54BB47B167E00E566
:10F12D00342536FFEE3533FE7B007A00793712FD3C
:10F13D00C7804E7E00E5342536FFEE3533FEC3EF36
:10F14D00940CEE9400500B7B007A00793712FDBAC7
:10F15D00802F7E00E5342536FFEE3533FEEF64203B
:10F16D004E700585BF378019EF642D4E7005854BA8
:10F17D0037800EEF64304E70058545378003753747
:10F18D0001AF3712FD20AF3712FD83053602F111A5
:10F19D00E534640A45337059FB7A007937FFFE1266
:10F1AD00FDBAAF3712FD20AF3712FD837B007A0019
:10F1BD0079377F017E0012FDBAAF3712FD20AF37D0
:10F1CD0012FD837B007A0079377F027E0012FDBA33
:10F1DD00AF3712FD20AF3712FD837B007A007937F0
:10F1ED007F037E0012FDBAAF3712FD20AF3712FD3F
:10F1FD008302F2AD7850E66410701BF53612FD19DE
:10F20D00744F2536F8E6FF12FD830536E536C394B7
:10F21D000640EA02F2AD7850E66419600302F2BED0
:10F22D0018E6FF12FD20784FE6FF12FD837850E6B9
:10F23D00FF12FD207850E6FF12FD83AF4812FD202E
:10F24D00AF4812FD837B007A007937E4FFFE12FD93
:10F25D00BAAF3712FD20AF3712FD837B007A0079EC
:10F26D00377F017E0012FDBAAF3712FD20AF371286
:10F27D00FD837B007A0079377F027E0012FDBAAFE5
:10F28D003712FD20AF3712FD837B007A0079377F6F
:10F29D00037E0012FDBAAF3712FD20AF3712FD838A
:10F2AD00784DE6FF12FD20784EE6FF12FD2012FE8E
:01F2BD00014F
:01F2BE00222D
:10F6BE007850E6640670527852E6FFB406087E0073
:10F6CE007854E6FD800E7852E6B40A137854E6FDBF
:10F6DE007F067E0012FDFA7854E6F54802F824788B
:10F6EE0052E6FFB410117E007854E6FD12FDFA7852
:10F6FE0054E6F54102F8247852E6642D600302F8D0
:10F70E00247854E6F54B02F8247850E66410600332
:10F71E0002F8247854E6F53B08E6FD7851E6FCFE47
:10F72E0008E6F97A002400F536EA3EF5358C39897B
:10F73E003AE53B6D7042F537F538C3E538953BE554
:10F74E00379400507874562538F8E6F534E536458A
:10F75E00357006E53845376012E5362538FFE53554
:10F76E003537FEAD3412FCA940012212FE010538D8
:10F77E00E53870C6053780C2E4F537F538C3E5388D
:10F78E00953BE53794005035E53825E02457F8E6EB
:10F79E00F534E53645357006E53845376012E53601
:10F7AE002538FFE5353537FEAD3412FCA940012270
:10F7BE0012FE010538E53870C4053780C00549E5ED
:10F7CE004964087051E54475F002A42411FFE5F078
:10F7DE0034EEFEE4FD12FCA9E54475F002A42412F9
:10F7EE00FFE5F034EEFEE4FD12FCA90544E5447598
:10F7FE00F002A42411FFE5F034EEFEAD3912FCA99F
:10F80E00E54475F002A42412FFE5F034EEFEAD3AA5
:10F81E0012FCA9E4F549E541B47F0CE4F549F54441
:10F82E0075417EF5298071E541B43F22E4F533AF91
:10F83E003312FD6B12FE010533E533C3947340EFB3
:10F84E0075413E75804CC2A0D2A1C2A2804AE5414C
:10F85E00B4330B12FE0112FDAA754134803AE54114
:10F86E00641F702C12FE017D1F7F107EEE12FCA90C
:10F87E007DF07F117EEE12FCA97DF07F127EEE12DE
:10F88E00FCA975411E75804CC2A0C2A1D2A28008EF
:09F89E00E541B4010312FE01D39F
:01F8A700223E
:08FDF200784E76FF1876FF221F
:10FD8300784DE66FFF90F2BF930866794DF7EF90D9
:04FD9300F3BF93F631
:01FD97002249
:08FC66008B3B8A3C893D8D3E79
:10FC6E00753F007540FF7DFFAF3E153EEF6026AB42
:10FC7E003B053DE53DAA3C7002053C14F912FAD253
:10FC8E006540FF90F2BF936D753F00F540EF90F326
:0AFC9E00BF93FD80D3E540FEEDFFAB
:01FCA8002239
:03FD670001080090
:10FD6B0075F65575F6AA75F65575BF04EF25E0F5D2
:08FD7B00F4E4F5F575F78222AE
:10FDAA0075F65575F6AA75F65575BF0475F783226B
:0BFDC7008F828E83E49312FAEB7F0121
:01FDD200220E
:07FDFA0074082FF8A6052292
:0DFDBA0074082FF8E612FAEB12FAD2FF22BD
:01F0000023EC
:10F2BF0000C1814001C0804101C0804100C1814037
:10F2CF0001C0804100C1814000C1814001C0804127
:10F2DF0001C0804100C1814000C1814001C0804117
:10F2EF0000C1814001C0804101C0804100C1814007
:10F2FF0001C0804100C1814000C1814001C08041F7
:10F30F0000C1814001C0804101C0804100C18140E6
:10F31F0000C1814001C0804101C0804100C18140D6
:10F32F0001C0804100C1814000C1814001C08041C6
:10F33F0001C0804100C1814000C1814001C08041B6
:10F34F0000C1814001C0804101C0804100C18140A6
:10F35F0000C1814001C0804101C0804100C1814096
:10F36F0001C0804100C1814000C1814001C0804186
:10F37F0000C1814001C0804101C0804100C1814076
:10F38F0001C0804100C1814000C1814001C0804166
:10F39F0001C0804100C1814000C1814001C0804156
:10F3AF0000C1814001C0804101C0804100C1814046
:10F3BF0000C0C101C30302C2C60607C705C5C40406
:10F3CF00CC0C0DCD0FCFCE0E0ACACB0BC90908C876
:10F3DF00D81819D91BDBDA1A1EDEDF1FDD1D1CDC66
:10F3EF0014D4D515D71716D6D21213D311D1D010D6
:10F3FF00F03031F133F3F23236F6F737F53534F4C6
:10F40F003CFCFD3DFF3F3EFEFA3A3BFB39F9F83835
:10F41F0028E8E929EB2B2AEAEE2E2FEF2DEDEC2C25
:10F42F00E42425E527E7E62622E2E323E12120E095
:10F43F00A06061A163A3A26266A6A767A56564A485
:10F44F006CACAD6DAF6F6EAEAA6A6BAB69A9A868F5
:10F45F0078B8B979BB7B7ABABE7E7FBF7DBDBC7CE5
:10F46F00B47475B577B7B67672B2B373B17170B055
:10F47F005090915193535292965657975595945445
:10F48F009C5C5D9D5F9F9E5E5A9A9B5B99595898B5
:10F49F00884849894B8B8A4A4E8E8F4F8D4D4C8CA5
:10F4AF004484854587474686824243834181804015
:0300000002F0010A
:0CF00100787FE4F6D8FD7581E402F04849
:10FAD200BB010689828A83E0225002E722BBFE0232
:09FAE200E32289828A83E4932265
:10FAEB00BB010689828A83F0225002F722BBFE01FA
:02FAFB00F322F4
:10FAFD00C2D5EC30E709B2D5E4C39DFDE49CFCEE24
:10FB0D0030E715B2D5E4C39FFFE49EFE12FB33C36D
:10FB1D00E49DFDE49CFC800312FB3330D507C3E468
:06FB2D009FFFE49EFE2292
:10FC1900AC1CAD1DAE1EAF1F7810EC4D4E4F7004DD
:10FC29007CA57DA5C3EC13FCED13FDEE13FEEF13CC
:10FC3900FF5010EC64CCFCED644CFDEE644EFEEF1D
:10FC490064CEFFD8DF8C1C8D1D8E1E8F1FEE547F56
:0DFC5900FE228E1C8F1D74A5F51EF51F22C6
:10F00D0002FB88E493A3F8E493A34003F68001F296
:10F01D0008DFF48029E493A3F85407240CC8C33304
:10F02D00C4540F4420C8834004F456800146F6DFD3
:10F03D00E4800B010204081020408090FD46E47E20
:10F04D00019360BCA3FF543F30E509541FFEE493C8
:10F05D00A360010ECF54C025E060A840B8E493A38F
:10F06D00FAE493A3F8E493A3C8C582C8CAC583CABA
:10F07D00F0A3C8C582C8CAC583CADFE9DEE780BE72
:01FD6A000098
:10FB3300BC000BBE0029EF8DF084FFADF022E4CCB6
:10FB4300F875F008EF2FFFEE33FEEC33FCEE9DEC7F
:10FB5300984005FCEE9DFE0FD5F0E9E4CEFD22EDC5
:10FB6300F8F5F0EE8420D21CFEADF075F008EF2F0F
:10FB7300FFED33FD4007985006D5F0F222C398FD00
:05FB83000FD5F0EA229D
:00000001FF
